:020000020000FC
:100000001CC011C010C00FC00EC00DC00CC00BC072
:100010000AC009C008C007C006C005C004C003C0AC
:1000200002C001C000C018955D9BFECF3CB9089589
:1000300032B73017E8F3F2BE089534E03EBF3FE533
:100040003DBF7894FF243FEF38BB33EC37BB3FE331
:1000500035BB30E334BBF2BA3CEF31BB30E838B9E2
:10006000F9BE35E033BFF2BE31E030BFF0BC3AE05C
:1000700042E039B94BB938E13AB93EE830BD4F2DCD
:10008000E199FECFFFBAFEBAE09A6DB373E088271C
:100090000AEFAD98CDDFAD9AAC98CADFAC9AC198A3
:1000A000C7DFC19AC098C4DFC09AC698C79801E05C
:1000B000BFDF1FE053B351275427512318E0C0E09E
:1000C000D0E0352F312351F028812395342F31236F
:1000D00011F4243010F4293C10F0412720E029933A
:1000E000169579F71FE0412735B342FB35F943FBFD
:1000F00034F935BB38B340FB30F941FB31F938BB3B
:100100004127342F617021F0337011F13CE003C0BE
:100110003C70F1F033E03423A9F0949A342F357019
:1001200061F0617029F040FF22C042FF08C01FC08B
:1001300042FF1DC040FF03C01AC08823C1F4609570
:100140008FEF15C0609590E0342F3A7009F09FEF63
:1001500090FF09C0342F3A7011F08FEF04C0342F94
:10016000357009F090E09498442309F48827617071
:10017000761729F1959AE199FECFFFBAFEBA6DBBC9
:10018000F894E29AE19A789404E152DF662351F000
:10019000C698979A4DDF97984BDF939A49DF9398CB
:1001A000C79A09C0C798969A43DF969841DF929AFA
:1001B0003FDF9298C69A0AEA3BDF9598762F77CF71
:00000001FF
